:10000000E9C9FBC9FAC9F9C9F8C9F7C9F6C9F5C9F7
:10001000F4C9F3C9F2C9F1C9F0C9EFC9EEC9EDC914
:10002000ECC9EBC9EAC9080808000000000000009C
:1000300000000000000000065F5F060000000007EF
:10004000070007070000147F7F147F7F1400242E11
:100050006B6B3A120000466630180C666200307A0C
:100060004F5D377A48000407030000000000001CC1
:100070003E63410000000041633E1C000000082A6E
:100080003E1C1C3E2A0808083E3E0808000000806E
:10009000E0600000000008080808080800000000F0
:1000A0006060000000006030180C060301003E7F15
:1000B0004149417F3E0040427F7F404000006273E3
:1000C00059496F660000226349497F360000181CB9
:1000D00016537F7F5000276745457D3900003C7EE1
:1000E0004B4979300000030371790F070000367F18
:1000F00049497F360000064F49693F1E0000000055
:100100006666000000000080E66600000000081C33
:1001100036634100000024242424242400000041EC
:1001200063361C080000020351590F0600003E7F91
:10013000415D5D1F1E007C7E13137E7C0000417FAD
:100140007F49497F36001C3E634141632200417F65
:100150007F41633E1C00417F7F495D416300417FD9
:100160007F491D0103001C3E6341517372007F7F74
:1001700008087F7F000000417F7F41000000307051
:1001800040417F3F0100417F7F081C776300417F32
:100190007F41406070007F7F0E1C0E7F7F007F7F5D
:1001A000060C187F7F001C3E6341633E1C00417FAC
:1001B0007F49090F06001E3F21717F5E0000417FCD
:1001C0007F09197F6600266F4D5973320000034185
:1001D0007F7F410300007F7F40407F7F00001F3F03
:1001E00060603F1F00007F7F3018307F7F004367D3
:1001F0003C183C674300074F78784F07000047637F
:1002000071594D677300007F7F4141000000010379
:10021000060C183060000041417F7F000000080C90
:100220000603060C080080808080808080800000AB
:10023000030704000000207454543C784000417FC0
:100240003F4848783000387C44446C2800003078BF
:1002500048493F7F4000387C54545C180000487E79
:100260007F490302000098BCA4A4F87C0400417FED
:100270007F08047C780000447D7D4000000060E041
:100280008080FD7D0000417F7F10386C440000417C
:100290007F7F400000007C7C18381C7C78007C7CD0
:1002A00004047C780000387C44447C38000084FCE2
:1002B000F8A4243C1800183C24A4F8FC8400447CD6
:1002C000784C041C1800485C54547424000000044A
:1002D0003E7F442400003C7C40403C7C40001C3C71
:1002E00060603C1C00003C7C7038707C3C00446CBE
:1002F0003810386C44009CBCA0A0FC7C00004C640E
:10030000745C4C64000008083E7741410000000026
:10031000007F7F0000004141773E08080000020393
:100320000103020301000000000000000000007C47
:100330007E13117F7F00007F7F4949793000007F65
:100340007F49497F3600007F7F0101010100C0FE27
:100350007F417FFEC000007F7F49494941006377AC
:100360001C7F7F1C776300226349497F3600007F32
:100370007F180C7F7F00007E7F190D7F7E00007F3D
:100380007F1C36634100007C7E03017F7F007F7FFE
:100390000E1C0E7F7F00007F7F08087F7F00003EDD
:1003A0007F41417F3E00007F7F01017F7F00007F12
:1003B0007F11111F0E00003E7F41416322000001AA
:1003C000017F7F01010000276F48487F3F000E1F1B
:1003D000117F7F111F0E0063771C1C776300007F65
:1003E0007F40407FFFC000070F08087F7F007F7FAE
:1003F000407F7F407F7F7F7F407F7F40FFFF017F87
:100400007F48487830007F7F4878307F7F00007FCA
:100410007F4848783000224149496B3E1C007F7F6D
:10042000083E7F417F3E004E7F31117F7F00207468
:1004300054543C78400000347E4A4A7A3000007CB4
:100440007C54547C2800007C7C0404040400C0F824
:100450007C447CFCC00000387C54545C1800446C24
:10046000387C7C386C4400286C44547C2800007C28
:100470007C30187C7C00007C7C321A7C7C00007C08
:100480007C10386C44000070780C047C7C007C7C10
:100490001838187C7C00007C7C10107C7C000038B4
:1004A0007C44447C3800007C7C04047C7C00007C20
:1004B0007C24243C180000387C44446C2800000450
:1004C000047C7C040400000C5C50507C3C00183C14
:1004D000247C7C243C1800446C38386C4400007C3C
:1004E0007C40407CFCC0000C1C10107C7C007C7CA0
:1004F000407C7C407C7C7C7C407C7C40FCFC047CA4
:100500007C50507020007C7C5070207C7C00007CF3
:100510007C505070200000445454547C38007C7C43
:1005200010387C447C3800487C34147C7C0000000B
:1005300000000000000000000000000000000000BB
:1005400000000000000000000000000000000000AB
:10055000000000000000000000000000000000009B
:10056000000000000000000000000000000000008B
:10057000000000000000000000000000000000007B
:10058000000000000000000000000000000000006B
:10059000000000000000000000000000000000005B
:1005A000000000000000000000000000000000004B
:1005B000000000000000000000000000000000003B
:1005C000000000000000000000000000000000002B
:1005D000000000000000000000000000000000001B
:1005E000000000000000000000000000000000000B
:1005F00000000000000000000000000000000000FB
:1006000000000000000000000000000000000000EA
:100610000000000FFFFFFFFFFFFFFFFFFFFFFFFFD7
:10062000FFFFFFFFFFFFFFFFFFFFFFFFFFFFFFFFDA
:10063000FFFFFFFFFFFFFFFFFFFFFFFFFFFFFFFFCA
:10064000FFFFFFFFFFFFFFFFFFFFFFFFFFFFFFFFBA
:10065000FFFFFFFFFFFFFFFFF000000000000FFFA4
:10066000000000FFFFFFFFFFFFFFFFFFFFFFFFFF97
:10067000FFFFFFFFFFFFFFFFFFFFFF999333000026
:10068000000000000000003003006003003003336E
:10069000CCCFFFFFFFFFFFFFFFFFFFFFFFFFFFFFCD
:1006A000FFFFFFF000000000000FFF300900FFFF18
:1006B000FFFFFFFFFFFFFFFFFFFFFFFFFFFFFFFF4A
:1006C000FFFFFF000000000000600C30C30C30C3CF
:1006D0000C30C30C30C30C30C30C30C30C3090034F
:1006E00033FFFFFFFFFFFFFFFFFFFFFFFFFFF000F4
:1006F000000000000999300000FFFFFFFFFFFFFF2F
:10070000FFFFFFFFFFFFFFFFFFFFFF33300000038E
:1007100000C30C30C30C30C30C30C30C30C30C30DE
:10072000C30C30C30C30C30C30C30C30C30300CC3B
:10073000CFFFFFFFFFFFFFFFFFF0000000000006FC
:1007400066000000FFFFFFFFFFFFFFFFFFFFFFFF4F
:10075000FFFFFFCCC000000000C30C30C30C30C34F
:100760000C30C30C30C30C30C30C30C30C30C30C82
:1007700030C30C30C30C30C30C30C30666FFFFFF20
:10078000CCCFFFFFF000000000000666000000FF75
:10079000FFFFFFFFFFFFFFFFFFFFFFFFF9990000D3
:1007A00000300C30C30C30C30C30C30C30C30C30E1
:1007B000C30C30C30C30C30C30C30C30C30C30C37B
:1007C0000C30C30C30C30C30333FFFFFF666FFF034
:1007D00000000000000666C30900FFFFFFFFFFFFE7
:1007E000FFFFFFFFFFFFCCC000000900C30C30C3B8
:1007F0000C30C30C30C30C30C30C30C30C30C30CF2
:1008000030C30C30C30C30C30C30C30C30C30C30BD
:10081000C30C30900333333999FFF000000000001F
:100820000666300300FFFFFFFFFFFFFFFFFFFFFF34
:10083000FF000000600C30C30C30C30C30C30C3020
:10084000C30C30C30C30C30C30C30C30C30C30C3EA
:100850000C30C30C30C30C30C30C30C30900C30CC4
:1008600030333CCCFFF00000000000066690090029
:10087000FFFFFFFFFFFFFFFFFFFFF000000300C3CC
:100880000C30C30C30C30C30C30C30C30C30C30C61
:1008900030C30C30C30C30C30C30C30C30C30C302D
:1008A000C30C30C30C30C30C30330C30900FFFFF3F
:1008B000F000000000000333600600FFFFFFFFFFB1
:1008C000FFFFFFFFCCC000000C30C30C30C30C3066
:1008D000C30C30C30C30C30C30C30C30C30C30C35A
:1008E0000C30C30C30C30C30C30C30C30C30C30C01
:1008F00030C30C30999C30300000FFF00000000045
:10090000000666300300FFFFFFFFFFFFFFFFFF0051
:100910000000600C30C30C30C30C30300C30C30C02
:1009200030C30C30C30C30C30C30C30C30C30C309C
:10093000C30C30C30C30C30C30C30C30300C3063EC
:100940003C30C303000000000000000006663003D6
:1009500000FFFFFFFFFFFFFFFCCC000000C30C30D7
:10096000C30C30600C30C30C30C30C30C30C30C32C
:100970000C30C30C30C30C30C30C30C30C30C30C70
:1009800030C30C30C30C30300C30C30C30000FFFC0
:10099000FFF000000000000666000000FFFFFFFF00
:1009A000FFFFFFF000000300C30C30C30000C30CC6
:1009B00030C30C30C30C30C30C30C30C30C30C300C
:1009C000C30C30C30C30C30C30C30C30C30C30C369
:1009D0000C30300C30C30C30000FFFFFF000000073
:1009E00000000666300600FFFFFFFFFFFFFFF0007C
:1009F000000C30C30C30000C30C30C30C309006055
:100A00000C30C30C30C30C30C30C30C30C30C30CDF
:100A100030C30C30C30C30C30C30C30C30300C303E
:100A2000C30C30333FFFFFF0000000000009999035
:100A30000C30FFFFFFFFFFFFCCC000300C30C300C5
:100A400000C30C30C30C30300C30C30C30C30C303E
:100A5000C30C30C30C30C30C30C30C30C30C30C3D8
:100A60000C30C30C30C30C30C30900C30C30666FAC
:100A7000FFFFF000000000000999600C30FFFFFF4D
:100A8000FFFFFF000000C30C30000C30C30C30C36C
:100A90000300C30C30C30C30C30C30C30C30C30C88
:100AA00030C30C30C30C30C30C30C30C30C30C301B
:100AB000C30C30C30999C30900CCCFFFFFF000007D
:100AC0000000000999600C30FFFFFFFFFFFF0000EE
:100AD00000000300C30C30C30C30300C30C30C30AA
:100AE000C30C30C30C30C30C30C30C30C30C30C348
:100AF0000C30C30C30C30C30C30C30C30C30C303F8
:100B000033C30900FFFFFFFFF00000000000099958
:100B1000300C30FFFFFFFFF999000000C30C30C319
:100B20000C30C30000C30C30C30C30C30C30C30CFA
:100B300030C30C30C30C30C30C30C30C30C30C308A
:100B4000C30C30C30C30C30C30C30C30C3060030B0
:100B50000FCCFFF000000000000CCC300C30FFFF89
:100B6000FFFFF333000000900C30C30C30000C305A
:100B7000C30C30C30C30C30C30C30C30C30C30C3B7
:100B80000C30C30C30C30C30C309003000303603C6
:100B9000903C03603603C0360300600CCCFFF000CD
:100BA000000000000CCC300C30FFFFFFFFF0000015
:100BB0000600000900300300C30C30C30C30C30C26
:100BC00030C30C30C30C30C30C30C30C30C30C30FA
:100BD0009000303C03C03C03C03C03903C03903386
:100BE00033C03C03C0360CCCFFF000000000000C0A
:100BF000CC600C30CCCFFFFFF000000C30C30900FC
:100C0000C30C30C30C30C30C30C30C30C30C30C326
:100C10000C30C30C30C30C303003903C03C03C0399
:100C2000C03C03C03C03C03C03C03C03C03C03C009
:100C3000030666FFF000000000000CCC600C309949
:100C40009FFFFFF000000C30C30C30C30C30C30C0E
:100C500030C30C30C30C30C30C30C30C30C30C3069
:100C60006003603C03C03C03C03C03C03C03C03C89
:100C700003C03C03903603900600303C0333FFF082
:100C800000000000000CCC600C30999FFFFFF000CA
:100C9000300C30C30C30C30C30C30C30C30C30C329
:100CA0000C30C30C30C30C30C306003C03C03C0303
:100CB000C03C03C03C03C03C03C03C03C03C0390A9
:100CC0003C03C03C03C0360666FFF0000000000095
:100CD0000CCC600C30CCCFFFFFF000600C30C30CAC
:100CE00030C30C30C30C30C30C30C30C30C30C30D9
:100CF000C30C30C300003C03C03C03C03C03C03CF9
:100D000003C03C03C03C03C03C03603C03C03C0345
:100D1000C0030999FFF000000000000CCC300C303B
:100D2000CCCFFFFFF000900C30C30C30C30C30C3AD
:100D30000C30C30C30C30C30C30C30C309000003AB
:100D4000C03C03C03C03C03C03C03C03C03C03C0E8
:100D50003C03903600300003C03C03C0000FFFFF8F
:100D6000F000000000000CCC300C30CCCFFFCCC029
:100D700000C30C30C30C30C30C30C30C30C30C3078
:100D8000C30C30C30C30C300303C03C03C03C03C38
:100D900003C03C03C03C03C03C03C03C03603603BB
:100DA000900000003C0360333FFFFFF000000000B4
:100DB000000CCC300C30999FFFCCC000C30C30C36A
:100DC0000C30C30C30C30C30C30C30C30C30C30C1C
:100DD000300003C03C03C03C03C03C03C03C03C024
:100DE0003C03C03C03C03C03C00300003C000000C7
:100DF0000000FFFFFFFFF000000000000CCC300CF3
:100E000030633FFFCCC000C30C30C30C30C30C3088
:100E1000C30C30C30C30C30C30C30C303903C03C9E
:100E200003C03C03C03C03C03C03C03C03C03C03C4
:100E3000C03C03C03903C03C0060000FFFFFFFFF50
:100E4000FFF000000000000CCC300C30333FFF9965
:100E50009000C30C30C30C30C30C30C30C30C30C37
:100E600030C30C30C300003C03C03C03C03C03C093
:100E70003C03C03C03C03C03C03C03C03C03C03C3B
:100E800003C0360000FFFFFFFFFFFFFFF000000080
:100E900000000CCC300C30000FFF666000C30C303B
:100EA000C30C30C30C30C30C30C30C30C30C30C384
:100EB00003903C03C03C03C03C03C03C03C03C0364
:100EC000C03C03C03C03C03C03C03C0030000CCC21
:100ED000FFFFFFFFFFFFFFF000000000000CCC3021
:100EE0000C30000FFF666000C30C30C30C30C30C25
:100EF00030C30C30C30C30C30C309003C03C03C073
:100F00003C03C03C03C03C03C03C03C03C03C039AD
:100F10000390360030000900000FFFFFFFFFFFFFC6
:100F2000FFFFF000000000000CCC300C30300FFF51
:100F3000666000C30C30C30C30C30C30C30C30C32C
:100F40000C30C30C303303C03C03C03C03C03C0333
:100F5000C03C03C03C03C0000C30C30C30C30C3099
:100F6000C30000666FFFFFFFFFFFFFFFFFF0000001
:100F70000000000CCC300C30300FFF666000C30C5A
:100F800030C30C30C30C30C30C30C30C30C30C3036
:100F90003C03C03C03C03C03C03C03C03C03C03C1A
:100FA0000390900C30C30C30C30600000CCCFFFF44
:100FB000FFFFFFFFFFFFFFFFF000000000000999A7
:100FC000300C30300FFF666000C30C30C30C30C3F0
:100FD0000C30C30C30C30C30C306003C03C03C03D0
:100FE000C03C03C03C03C03C03C03C03900006006F
:100FF000600000000CCCFFFFFFFFFFFFFFFFFFFFC3
:10100000FFFFFFF000000000000666300C30300CDF
:10101000CC333000C30C30C30C30C30C30C30C30A5
:10102000C30C30C303603C03C03C03C03C03C03C62
:1010300003C0030000000000000000333FFFFFFF7B
:10104000FFFFFFFFFFFFFFFFFFFFFFFFFFFFF000BE
:10105000000000000666300C30600333333000C3FC
:101060000C30C30C30C30C30C30C30C30C30300315
:10107000C03C03C03C03C03C0390000000300900AA
:10108000C30C30C30900000999FFFFFFFFFFFFFFFA
:10109000FFFFFFFFFFFFFFFFFFF000000000000960
:1010A00099000C30900000000000C30C30C30C30DD
:1010B000C30C30C30C30C309003903C03C03C03C2F
:1010C0000000000300C30C30C30C30C30C30C30C51
:1010D00030C30C30900000999FFFFFFFFFFFFFFF20
:1010E000FFFFFFFFF000000000000999000C3090A6
:1010F0000000000000C30C30C30C30C30C30C30C24
:1011000030C300003C03C03C0390000C30C30C30E3
:10111000C30C30C30C30C30C30C30C30C30C30C311
:101120000C30C30600000999FFFFFFFFFFFFFFF02F
:1011300000000000000999000C30C300000000000E
:10114000C30C30C30C30C30C30C30C300003903CD4
:1011500003C03C0000C30C30C30C30C30C30C30CC4
:1011600030C30C30C30C30C30C30C30C30C30C3054
:10117000C30C30300000FFFFFFFFF0000000000054
:101180000CCC000C30C30000000300C30C30C30CB7
:1011900030C30C30C30000360360390360360900E9
:1011A000C30C30C30C30C30C30C30C30C30C30C381
:1011B0000C30C30C30C30C30C30C30C30C30C30C28
:1011C00030600CCCFFF000000000000CCC000C30B4
:1011D000C30300000C30C30C30C30C30C30C300010
:1011E0000000030030360360000C30C30C30C30C29
:1011F00030C30C30C30C30C30300000000000000FB
:10120000300600900C30C30C30C30900600999FF10
:10121000F000000000000CCC000C30C30C30C30CFC
:1012200030C30C30C30C30C30C30C30C30C30C3093
:10123000000030300C30C30C30C30C30C30C30C352
:101240000C30C30600600300300000000000666C34
:10125000CC999000600900000FFFFFF00000000033
:10126000000CCC000900C30C30C30C30C30C30C3DD
:101270000C30C30C30C30C30C30C30C30C30300CFA
:1012800030C30C30C30C30C30C30C30C30C30C3033
:10129000C30C30C30C30C30C30C30930600000995C
:1012A0009FFFFFFFFFFFF000000000000FFF0003A3
:1012B00000C30C30C30C30C30C30C30C30C30C3033
:1012C000C30C30C30C30C30C30C30C30C30C30C360
:1012D0000C30C30C30C30C30C30C30C30C30C30C07
:1012E00030C30C30C30C30C30C30900000FFFFFF44
:1012F000FFF000000000000FFF000000600C30C392
:101300000C30C30C30C30C30C30C30C30C30C30CD6
:1013100030C30C30C30C30C30C30C30C306006003B
:10132000000000000000000600600900C30C30C38C
:101330000C30C30600C30000FFFFFFFFF0000000F9
:1013400000000FFFCCC00000000000000000030000
:10135000300600900900900C3090060060030000F9
:10136000000000000000000000000000000000007D
:101370000000000000000000000000000030090034
:10138000900000FFFFFFFFF00000000000000000E1
:10139000000000000000000000000000000000004D
:1013A000000000000000000000000000000000003D
:1013B000000000000000000000000000000000002D
:1013C000000000000000000000000000000000001D
:1013D0000000000011241FBECFE5D4E0DEBFCDBF6A
:1013E00011E0A0E6B0E0E2E2FCE102C005900D925F
:1013F000AC32B107D9F797D312C402C6A998AB98FB
:101400008823A9F0AA9AAB9A90E021E009C0AA9893
:10141000AB9A822F8A95F1F79F5F983031F0660F73
:10142000AB9867FFF4CFAA9AF3CFA99A0895AA9828
:10143000EACF0F931F93182F062F80E06BE2DEDFB9
:1014400081E0612FDBDF81E0612FD8DF80E06AE29D
:10145000D5DF81E0602FD2DF81E0602FCFDF1F91E9
:101460000F9108950F931F938A01E3DF80E06CE2F0
:10147000C5DFA998B80175956795759567957595B8
:1014800067957595679581E0B9DF02951295107F94
:101490001027007F102781E0602FB0DFA99A80E03D
:1014A00060E0ACDF1F910F9108952F923F924F9211
:1014B0005F926F927F928F929F92AF92BF92CF92E4
:1014C000DF92EF92FF920F931F93CF93DF93A82E9B
:1014D000B62E242E322E480130E0261B3109842FEF
:1014E00090E08A19910937FD68C071E0472E512CB0
:1014F00097FD5CC061E0662E712C6901CC0CDD1C8F
:101500007C01EE0CFF1C8A2D6B2DA401ABDFCE14E9
:10151000DF047CF52A14D1F0C70195958795E60183
:10152000C81BD90B062D162D1A0D02C0CC0DDD1DC2
:10153000D7FD03C0B40CCE19DF09812F6B2DA40198
:1015400091DF100F812F801B281681F7DF91CF913B
:101550001F910F91FF90EF90DF90CF90BF90AF90D1
:101560009F908F907F906F905F904F903F902F90C3
:1015700008953B1459F3C60195958795E701C81B5B
:10158000D90B042D142D1B0D02C0CE0DDF1DD7FD70
:1015900003C0A60CCC19DD098A2D612FA40162DFDE
:1015A000100F812F801B381681F7D0CF9095819531
:1015B0009F4F66246A94762CA0CF309521953F4F9B
:1015C00044244A94542C94CF9F92AF92BF92CF92CE
:1015D000DF92EF92FF920F931F93CF93DF93D82E5A
:1015E000A62EC42EB22E0130F1F02A2D87015DDF28
:1015F0008D2D6B2D4C2D2B2D58DF8D2D6A2D4D2DC6
:101600002B2D53DF8C2D6A2D4C2D2B2D4EDFDF9192
:10161000CF911F910F91FF90EF90DF90CF90BF90EF
:10162000AF909F900895942E841708F475C00C2DE8
:10163000CD1408F46BC0DB2CAB1408F461C01B2D77
:10164000BA1408F45BC080E06BE2D8DE81E0692D5B
:10165000D5DE81E0602FD2DE80E06AE2CFDE81E07D
:101660006D2DCCDE81E0612FC9DE80E06CE2C6DE4C
:10167000212F30E02F5F3F4F2D193109802F90E04F
:10168000019689199109289FA001299F500D389F23
:10169000500D112457FD46C06A01D594C794D7FC5C
:1016A00029C0C701959587959595879595958795B7
:1016B00095958795082F8F2D992787FD9A95182F37
:1016C0001F70C70182959295907F9827807F9827F9
:1016D000182BC0E0D0E0A99881E0602F8FDE81E078
:1016E000612F8CDE81E06E2D89DEA99A2196CC16C1
:1016F000DD068CF780E060E081DE89CF1A2DA3CF74
:10170000DA2C1B2DBA1408F09ECFF8CF0D2DDB2C50
:10171000AB1408F094CFF4CF982E0C2DCD1408F014
:101720008ACFF4CF4F5F5F4FB7CFEF92FF920F9307
:1017300084B38F6084BBA998AA98AB9AA89AA898FA
:1017400080E49CE9FC013197F1F7A89A0197F1F741
:10175000AB9AAA9AAB9A80E061E050DE80E061E14A
:101760004DDE80E063E04ADE80E29EE40197F1F71F
:1017700080E069E243DE80E063E140DE80E06BE22E
:101780003DDE81E060E03ADE81E063E837DE80E064
:101790006AE234DE81E060E031DE81E063E82EDE83
:1017A00080E197E20197F1F780E06CE227DE24EF19
:1017B00031E048EC50E0CA010197F1F72150304088
:1017C000D1F780E060E21ADE80E06AE317DE81E0B4
:1017D00063E014DE80E066E311DE81E060E00EDEAF
:1017E00080E065E20BDE81E06DE208DE80E068E229
:1017F00005DE80E060E043E823E801E0EE24FF241A
:10180000E3DE80E069E2FADD0F91FF90EF9008954A
:101810004F925F927F928F929F92AF92BF92CF92A0
:10182000DF92EF92FF920F931F93CF93DF93782E67
:10183000A62EF42EE901642F6A0DA90113DE6A2D8C
:101840006F19872DAE010EDE8F2D870D6A2DAE012B
:1018500009DE872D8F196A2DAE0104DEFF2009F401
:1018600056C08F2D90E021E0C22ED12CC81AD90A83
:10187000880F991F44245524481A590ABF2CEE2476
:1018800013E0812E912C06C0C80CD91C82E090E098
:10189000880E991ED7FC07C0BA9482E090E0480EEB
:1018A000591EC40CD51CE394FE2CF70C1B2D1A0DED
:1018B0008F2D612FAE01D6DD072D0E19802F612FE0
:1018C000AE01D0DD1A2D1B198F2D612FAE01CADD9F
:1018D000802F612FAE01C6DDFB2CF70C1E2D1A0DDB
:1018E0008F2D612FAE01BEDD072D0B19802F612FCB
:1018F000AE01B8DD1A2D1E198F2D612FAE01B2DD9C
:10190000802F612FAE01AEDDEB1408F4BDCFDF9167
:10191000CF911F910F91FF90EF90DF90CF90BF90EC
:10192000AF909F908F907F905F904F9008952F92EF
:101930003F924F925F926F927F928F929F92AF925F
:10194000BF92CF92DF92EF92FF920F931F93DF939C
:10195000CF9300D00F92CDB7DEB7982FA62E498334
:101960002901380187FD5FC0E6E2F0E08491282E6E
:10197000332431968491C82EDD243196249121148C
:101980003104C1F1892F90E04F9730E0829F4001F0
:10199000839F900C929F900C112486E290E0880E19
:1019A000991EEE24FF24F401EE0DFF1DB490C11426
:1019B000D104D1F009810E0D10E81B821A820FC0EC
:1019C000A3018A2D9A81891B602F4CDDEA81FB815E
:1019D0003196FB83EA83EC15FD0530F41695812FD3
:1019E0008B2171F3A201EDCF0894E11CF11CE214EC
:1019F000F304C8F280E060E001DD0F900F900F90DB
:101A0000CF91DF911F910F91FF90EF90DF90CF90DA
:101A1000BF90AF909F908F907F906F905F904F900E
:101A20003F902F90089590549FCFAF92BF92CF9246
:101A3000DF92EF92FF920F931F93CF93DF93EC010E
:101A4000E62EF42E5901680103C0219688E0F80EB5
:101A50008881882341F06E2D4F2D9501860167DF27
:101A600083E88E1590F7DF91CF911F910F91FF9032
:101A7000EF90DF90CF90BF90AF900895CF92DF921C
:101A8000EF92FF920F931F93CF93DF93F82EE62EE2
:101A9000C42ED22E80E06BE2B1DC81E06F2DAEDC93
:101AA000FA94FC0C81E06F2DA9DC80E06AE2A6DCF0
:101AB00081E06E2DA3DCEA94ED0C81E06E2D9EDCBE
:101AC00080E06CE29BDCDC9C70011124F594E794CF
:101AD0001E141F04E4F4C0E0D0E0A998F80164915A
:101AE00081E08CDC0F5F1F4FF801649101501040C2
:101AF00081E084DCF80132960D5F1F4FE49181E0B4
:101B00006E2F7CDCA99A2196CE15DF0534F380E098
:101B100060E074DCDF91CF911F910F91FF90EF9007
:101B2000DF90CF900895EF92FF920F931F93FDDD0A
:101B300080E690E06AE043E020EF30E000E010E073
:101B400074DF81E790E064E143E020EF30E06DDF97
:101B500082E890E06EE143E020EF30E066DF83E969
:101B600090E068E243E020EF30E05FDF84EA90E05D
:101B700062E343E02FEF3FE058DF85EB90E06CE35A
:101B800043E02FEF3FE051DF86EC90E066E443E076
:101B90002FEF3FE04ADF87ED90E060E543E02FEF75
:101BA0003FE043DF88EE90E06AE543E020E03FE07D
:101BB0003CDF89EF90E064E643E02FEF3FE035DF64
:101BC0008AE091E06EE643E02FE030E02EDF8BE12B
:101BD00091E068E743E02FE030E027DF20E23EE4D9
:101BE00048EC50E0CA010197F1F721503040D1F79D
:101BF00080E060E043E823E801E05FE0E52EF12CBF
:101C0000E3DC89E269E242E322E30EE215E036DF3B
:101C100080E090E01F910F91FF90EF900895F8946D
:021C2000FFCFF4
:101C22004142434445464748494A4B4C4D4E4F502A
:101C32000052535455565758595A202020202020DC
:101C420020006162636465666768696A6B6C6D6EC9
:101C52006F700072737475767778797A20202020FD
:101C620020202000C0C1C2C3C4C5C6C7C8C9CACBD0
:101C7200CCCDCECF00D0D1D2D3D4D5D6D7D8D9DA05
:101C8200DBDCDDDEDF00E0E1E2E3E4E5E6E7E8E914
:101C9200EAEBECEDEEEF00F0F1F2F3F4F5F6F7F823
:101CA200F9FAFBFCFDFEFF0020CFD0C8C2C5D2204E
:101CB200CCC8D020212121200020202031323334F1
:101CC20035363738393020202000213F4023242563
:101CD200267B7D5B5D2E2C3A3B2A005E28295F2BFA
:0C1CE2002D3D7E7C3C2F3E202020200069
:00000001FF
